:1000000019C018951895189518951895189518955C
:10001000189518951895189518955AC21895189509
:1000200091C21895189518951895189518951895C2
:10003000189518958FEF8DBFC8EDE0EC4E2E82E03D
:100040008EBFD2E0F2E05F2EA89584B7082E877F9E
:1000500084BF88E199278093600090936000EEEF61
:10006000F1E0A0E0B1E088278D933197E9F704D360
:100070006624D7D28CE053D3EEECF8E0CCD2E1E0AA
:10008000F0E0F1D2519852985398599A5A9A5B9A43
:1000900080E08093800086E08093810085E085BDCC
:1000A00080E084BD882785BD76E076BD7894709128
:1000B0006F00716070936F0070916E00716070934B
:1000C0006E0080918100887F80938100AAD28FE7A3
:1000D00012E0BAD2E0EEF8E09ED28FEB14E0B4D298
:1000E000E8EEF8E098D280E090E09093850080936D
:1000F000840085E085BD86E080938100A9E0B1E0C1
:100100008C9187FB0EF0E3C1A0E0B1E00D911D9151
:100110002D913C9140E050E061E070E03BD3A0E0E5
:10012000B1E00D931D932D933D93A4E8B0E08D9124
:100130009C91A4E0B1E08D939D9388278D938C933F
:1001400080E090E09093850080938400A0E0B1E08F
:100150000D911D912D913C91A4E0B1E04D915D91E7
:100160006D917C913ED3A0E0B1E00D931D932D9352
:100170003D93499927C04A9912C0A0E0B1E00D9182
:100180001D912D913C9148EF51EA61E070E029D337
:10019000A0E0B1E00D931D932D933D9313C04B99B7
:1001A00011C0A0E0B1E00D911D912D913C9146EC64
:1001B00051E160E070E015D3A0E0B1E00D931D9334
:1001C0002D933D93499B27C04A9912C0A0E0B1E00E
:1001D0000D911D912D913C9148EF51EA61E070E045
:1001E00005D3A0E0B1E00D931D932D933D9313C073
:1001F0004B9911C0A0E0B1E00D911D912D913C9162
:1002000046EC51E160E070E0F1D2A0E0B1E00D9386
:100210001D932D933D9300E010E020E030E0A4E03A
:10022000B1E00D931D932D933C934FE057E260E0B6
:1002300070E0A0E0B1E00D911D912D913C91DBD2D9
:1002400014F009F001C015C0A4E0B1E0CFD1A0E0E6
:10025000B1E00D911D912D913C9140E157E260E09C
:1002600070E0C4D2A0E0B1E00D931D932D933D93B7
:10027000DCCF8FE711E0E8D141E050E060E070E0D2
:10028000A4E0B1E00D911D912D913C91B4D20CF4FC
:1002900001C004C0ECEEF8E0BED105C144E650E078
:1002A00060E070E0A4E0B1E00D911D912D913C91D2
:1002B000A2D20CF401C082C04AE050E060E070E0DD
:1002C000A0E0B1E00D911D912D913C9194D20CF4E0
:1002D00001C016C0E8EFF8E09ED1A8EAB2E0E4E081
:1002E000F1E09FD290D1EAEFF8E095D1A8EAB2E030
:1002F000E0E0F1E096D287D1E0E0F9E08CD15DC09A
:1003000044E650E060E070E0A0E0B1E00D911D91A6
:100310002D913C9170D20CF401C016C0E8EFF8E0CA
:100320007AD1A8EAB2E0E4E0F1E07BD26CD1E4E07B
:10033000F9E071D1A8EAB2E0E0E0F1E072D263D175
:10034000E0E0F9E068D139C048EE53E060E070E0E9
:10035000A0E0B1E00D911D912D913C914CD20CF497
:1003600001C016C0E8EFF8E056D1A8EAB2E0E4E038
:10037000F1E057D248D1E8E0F9E04DD1A8EAB2E087
:10038000E0E0F1E04ED23FD1E0E0F9E044D115C029
:10039000E8EFF8E040D1A8EAB2E0E4E0F1E041D2D1
:1003A00032D1ECE0F9E037D1A8EAB2E0E0E0F1E0E8
:1003B00038D229D1E0E0F9E02ED175C04AE050E012
:1003C00060E070E0A0E0B1E00D911D912D913C91B5
:1003D00012D20CF401C013C0A8EAB2E0E4E0F1E0EC
:1003E00020D211D1EAEFF8E016D1A8EAB2E0E0E0BD
:1003F000F1E017D208D1E0E0F9E00DD154C044E6B5
:1004000050E060E070E0A0E0B1E00D911D912D9111
:100410003C91F1D10CF401C013C0A8EAB2E0E4E0D1
:10042000F1E0FFD1F0D0E4E0F9E0F5D0A8EAB2E0E5
:10043000E0E0F1E0F6D1E7D0E0E0F9E0ECD033C065
:1004400048EE53E060E070E0A0E0B1E00D911D9156
:100450002D913C91D0D10CF401C013C0A8EAB2E0B8
:10046000E4E0F1E0DED1CFD0E8E0F9E0D4D0A8EAD2
:10047000B2E0E0E0F1E0D5D1C6D0E0E0F9E0CBD0E9
:1004800012C0A8EAB2E0E4E0F1E0CBD1BCD0ECE0ED
:10049000F9E0C1D0A8EAB2E0E0E0F1E0C2D1B3D027
:1004A000E0E0F9E0B8D000E010E020E030E0A0E0CB
:1004B000B1E00D931D932D933C93709109017F77CB
:1004C0007093090185E085BD86E08093810016CE9A
:1004D0000F921F922F923F924F925F927F92AF9214
:1004E000BF920F931F932F933F934F935F936F93FD
:1004F0007F938F939F93AF93BF93CF93DF93EF93AC
:10050000FF938FB78F93A0E0B1E070D08F918FBF32
:10051000FF91EF91DF91CF91BF91AF919F918F911B
:100520007F916F915F914F913F912F911F910F910B
:10053000BF90AF907F905F904F903F902F901F9013
:100540000F9018950F921F922F923F924F925F92A9
:100550007F92AF92BF920F931F932F933F934F932E
:100560005F936F937F938F939F93AF93BF93CF933B
:10057000DF93EF93FF938FB78F93A8E0B1E08C9157
:100580008F5F8C9300910801023309F00FC08091B6
:100590008100887F8093810080E080930801882714
:1005A00085BD7091090170687093090176E076BD90
:1005B0008F918FBFFF91EF91DF91CF91BF91AF915D
:1005C0009F918F917F916F915F914F913F912F916B
:1005D0001F910F91BF90AF907F905F904F903F9091
:1005E0002F901F900F901895F894FFCF0D911D91AB
:1005F0002D913C910F5F1F4F2F4F3F4F3C932E93F8
:100600001E930E930895A8EAB2E08D91882311F00D
:1006100075D0FBCF0895E1D0802D11F06FD0FBCFC6
:10062000089581E07CD025D080E879D08827809318
:100630000A0108958FE7213039F08FEB223021F045
:1006400083E9233009F083ED810F87FF08C083FF22
:1006500006C0804C282F204420930A0103C0204864
:1006600020930A015CC088EE93E085D03197D9F7DA
:10067000089583E099277FC08AEF90E07CD03C9A70
:100680003B9A3D9A3A9A399A389A409885E090E098
:1006900072D0419844984398459A429A419AEF9370
:1006A000FF93E0EFF1E05BD0FF91EF91419860D0D4
:1006B000419AEF93FF93E0EFF1E051D0FF91EF917A
:1006C000419856D0419AEF93FF93E0EFF1E047D085
:1006D000FF91EF9141984CD04298419AEF93FF934C
:1006E000E0EFF1E03CD0FF91EF91419841D088E2FA
:1006F00016D08EE014D086E012D0089590910A01B1
:10070000939590930A01993021F48F9380EC07D050
:100710008F91409A829505D004D02AD008954098B0
:10072000F9CF859510F4429A01C04298859510F44E
:10073000459A01C04598859510F4439A01C04398A5
:10074000859510F4449A01C04498419AEF93FF9321
:10075000E0EFF1E004D0FF91EF91419808953197D7
:10076000F1F70895689462F80895E89462F808959E
:1007700081E090E000C0EF93FF93EE27E82BE92B98
:1007800031F0E8E8F3E13197F1F70197D1F7FF9104
:10079000EF9108950F921F922F92C801D901489F9F
:1007A00080014A9F90014B9F202C499F100D211DD5
:1007B000321D5A9F202C589F100D211D321D599F0C
:1007C000200D311D689F200D311D699F300D789FD0
:1007D000300D2F901F900F900895C89531960020EE
:1007E0000895040F151F261F371F0895041B150BAE
:1007F000260B370B089504171507260737070895AA
:10080000000F111F221F331F08950095109520958A
:1008100030950F5F1F4F2F4F3F4F0895019110816B
:100820000EC001911191219130810BC00191108175
:1008300017FF05C03FEF2FEF04C0008111272227CB
:10084000332737FF03C0E1DF8DE28D93CF93DF9332
:10085000CF92DF92EF92AA24BB24CC24DD24EE2495
:1008600040E2CAE0DD2755E093E38881890F87FDE8
:100870009F7083FD907F891B89935A95A9F7C0DFEC
:10088000AA1CBB1CCC1CDD1CEE1C4A9551F7E8943D
:10089000EFE0FF2782910ED0EB30E0F71EF0689476
:1008A0008A2D0CD088278D93EF90DF90CF90DF9129
:1008B000CF910895982F829501D0892F8F70805DF8
:1008C00026F0803309F4089568948D93089577771E
:1008D000772E6E6F76612D746563682E68750000E3
:1008E000302E3030303000004D487A0020302E302D
:1008F000303030202020000020002E30303000002A
:0E090000202000002E3030002E3000002E008F
:00000001FF
